:100000004EC08CC065C064C063C062C061C060C0C7
:100010005FC05EC05DC05CC05BC05AC059C058C004
:1000200057C056C055C000CDD914F13C28E5A16C8D
:1000300078B5509D894416034A0075006C0069002C
:1000400065006E0020005600640047002003440055
:1000500061006E00270073002000410075006400FD
:1000600069006F0020004D00750078000A03300021
:1000700030003000310012010101FF000008666607
:1000800001000601010203010902120001010080C2
:10009000320904000000FF000000040309041124D9
:1000A0001FBECFEDCDBF10E0A0E6B0E0E6E0F6E089
:1000B00002C005900D92A236B107D9F710E0A2E672
:1000C000B0E001C01D92AF38B107E1F776D299C216
:1000D00097CFDC019FEF8FEF46E2F0E018C02D9143
:1000E0008227E82FEF70E40F3591E82FE295892FF2
:1000F000932F3170E327EF709295392F9F70307EE8
:100100008327E40F359193273170932783276A95CE
:1001100032F7809590958D939D9308950F931F933B
:100120002F93DF93CF930FB70F938299FECF8299CE
:100130000BC0829909C0829907C0829905C0829933
:1001400003C000E40ABFACC0C0917700DD27C858E7
:10015000DF4F0BE01CE024E0829BE9CF3F934F93FD
:100160006F9360B330E803C060B3432B49934427D7
:100170006C702627215020B32C70A9F137953C3F95
:10018000A0F56227615060B36C7037953C3F98F5DD
:1001900026272150379520B32C703C3F90F56227DD
:1001A000615037953C3F60B36C70A0F52627215015
:1001B00037953C3FC8F520B32C70622761503795C6
:1001C0003C3FB0F50A9560B37AF06C702627215059
:1001D00037953C3F88F520B32C70622761503795E6
:1001E0003C3F10F22DC031C052C0612720B32C70AB
:1001F0003F774160C6CF3F77426060B36C70212784
:10020000C7CF3F774460612720B32C7062276150CD
:100210003795C8CF3F7748602127316060B36C7055
:10022000262721503795C6CF3F7740616127C1CF40
:100230003F7740622127C4CF3F7740646127C9CF11
:100240003F774068212700C08FCF30E43ABF0B5082
:100250000195C01BD040288121FD2DC019811F7739
:1002600040918E00141799F4293691F4009168009A
:100270000023F1F0409176004423D1F440936800CC
:100280004091740040938E00C9E6D0E02BC0222735
:10029000209362006F914F913F910AB706FD45CFC1
:1002A0000F910FBFCF91DF912F911F910F91189553
:1002B000C1E6D0E016C0217059F3209162002223DC
:1002C00039F340917600442399F700937600209308
:1002D0007500009177004BE0401B40937700C0E62B
:1002E000D0E001E022B3237F286011B31C6022BB61
:1002F00011BB1CE030E830FF212722BB3795479522
:100300004C3FC0F530FF2127379522BB47954C3F26
:10031000A8F530FF21273795000022BB47954C3FB9
:1003200078F530FF21273795000022BB47954C3FD9
:1003300048F530FF2127699122BB379547954C3FFF
:1003400018F530FF2127379522BB47954C3F00F524
:1003500030FF21273795479522BB4C3FD8F430FF1B
:1003600021273795362F479522BB4C3FA8F40A9595
:1003700012F614C02127442722BBC2CF2127C5CFA4
:100380002127CBCF2127D1CF2127442722BBD7CF6D
:100390002127DACF2127DFCF2127E5CF237F22BBFB
:1003A0006F914F913F9100E40ABFDF91CF9111B35C
:1003B000022F286022BB137FDFBFDF912F91000047
:1003C00011BB02BB1F910F91189585B7836085BF44
:1003D0008BB780648BBF8D9A969A8E9A7894089585
:1003E0001F93CF93DF9380917600882309F473C025
:1003F0009091770081E080936300809175008D3249
:1004000011F010E05FC0CCE0D0E0C91BD109C858A2
:10041000DF4F1E818F8181111FEF8881807609F067
:1004200048C08981882321F41882198282E043C060
:10043000853029F48A8180937400959AA1C0863012
:1004400069F582E0809363008B81813021F482E141
:10045000C6E7D0E030C0823021F482E1C8E8D0E0C5
:100460002AC0833009F08CC08A81882321F484E07B
:10047000CAE9D0E020C0813021F486E1C6E3D0E0B3
:100480001AC0823021F480E2CCE4D0E014C0833082
:1004900009F076C08AE0CCE6D0E00DC0883019F4CF
:1004A00081E0888308C08A3009F06AC0188281E040
:1004B00002C0CE016BD0181708F0182FD093660039
:1004C000C09365001093640083EC809369001092E0
:1004D00068001092760080916800882309F043C07C
:1004E00040916300442309F43EC08091690098E87C
:1004F00089278093690090916400993010F018E08A
:1005000005C0992311F410E022C0192F2091650035
:1005100030916600413051F4F901AAE6B0E08191D2
:100520008D938E2F821B8117D0F30AC0F901AAE6A2
:10053000B0E0849131968D938E2F821B8117C8F382
:10054000F0936600E0936500911B909364008AE647
:1005500090E0612FBEDD1D5F1093680013501830CE
:1005600011F0109263008AE002C0815019F0839B61
:10057000FCCF08C01092740010928E00959802C0B3
:1005800080E09BCFDF91CF911F910895FC01818185
:10059000882311F488E00895813029F48091670060
:1005A000808381E00895823011F080E00895828197
:1005B00081708093670080E008951F93C398C29A6A
:1005C00087B38C6087BB87B38C7F87BB88B383601E
:1005D00088BB10926700F9DE11E002DFB09903C01A
:1005E0001092670004C0B19902C010936700809117
:1005F0006700882319F0C298C39AEFCFC398C29AB4
:06060000ECCFF894FFCFDF
:02060600D25AC6
:00000001FF
